:0200000480007A
:100000006F00C004732F2034930F8000630AFF0336
:10001000930F90006306FF03930FB0006302FF038A
:10002000170F0080130F0FFE63040F0067000F000F
:10003000732F203463540F006F004000136E9E53E3
:10004000171F00002320CFFD6FF09FFF732540F1A5
:100050006310050073251030635805000F00F00F82
:10006000130E100073000000130E00009702000032
:10007000938282F973905230735020307350303035
:1000800073504030970200809382C2F7638C020065
:10009000739052109302B01A739022307323203061
:1000A000E39E62F873500030970200009382420191
:1000B00073901234732540F17300203093001000C8
:1000C00013010000B3912000930E1000130E2000C6
:1000D000639ED1539300100013011000B3912000D0
:1000E000930E2000130E30006392D1539300100042
:1000F00013017000B3912000930E0008130E40000E
:100100006396D151930010001301E000B3912000D9
:10011000B74E0000130E5000639AD14F93001000A9
:100120001301F001B3912000B70E0080130E6000A0
:10013000639ED14D9300F0FF13010000B3912000A6
:10014000930EF0FF130E70006392D14D9300F0FFF9
:1001500013011000B3912000930EE0FF130E8000F6
:100160006396D14B9300F0FF13017000B391200010
:10017000930E00F8130E9000639AD1499300F0FF9C
:100180001301E000B3912000B7CEFFFF130EA000D3
:10019000639ED1479300F0FF1301F001B39120005B
:1001A000B70E0080130EB0006392D147B720212113
:1001B0009380101213010000B3912000B72E21216B
:1001C000938E1E12130EC0006392D145B7202121D9
:1001D0009380101213011000B3912000B74E4242D9
:1001E000938E2E24130ED0006392D143B720212189
:1001F0009380101213017000B3912000B79E90906D
:10020000938E0E08130EE0006392D141B720212196
:10021000938010121301E000B3912000B74E4848BC
:10022000130EF0006394D13FB72021219380101268
:100230001301F001B3912000B70E0080130E0001EE
:100240006396D13DB720212193801012130100FC49
:10025000B3912000B72E2121938E1E12130E100190
:100260006396D13BB720212193801012130110FC1B
:10027000B3912000B74E4242938E2E24130E2001DC
:100280006396D139B720212193801012130170FC9D
:10029000B3912000B79E9090938E0E08130E3001FC
:1002A0006396D137B7202121938010121301E0FC0F
:1002B000B3912000B74E4848130E40016398D135E2
:1002C0009300100013017000B3902000930E0008FB
:1002D000130E6001639CD033930010001301E00003
:1002E00033912000B74E0000130E70016310D1331C
:1002F00093003000B3901000930E8001130E800124
:100300006396D031130200009300100013017000B7
:10031000B391200013830100130212009302200006
:10032000E31452FE930E0008130E90016310D32FB6
:1003300013020000930010001301E000B3912000AD
:100340001300000013830100130212009302200027
:10035000E31252FEB74E0000130EA0016318D32B18
:1003600013020000930010001301F001B39120006C
:100370001300000013000000138301001302120099
:1003800093022000E31052FEB70E0080130EB0015E
:10039000631ED327130200009300100013017000A6
:1003A000B39120001302120093022000E31652FEC4
:1003B000930E0008130EC001639AD12513020000AA
:1003C000930010001301E00013000000B39120001F
:1003D0001302120093022000E31452FEB74E0000F5
:1003E000130ED0016394D123130200009300100078
:1003F0001301F0011300000013000000B39120006E
:100400001302120093022000E31252FEB70E008086
:10041000130EE001639CD11F130200009300100033
:100420001300000013017000B391200013021200AA
:1004300093022000E31452FE930E0008130EF00105
:100440006396D11D130200009300100013000000FA
:100450001301E00013000000B3912000130212000A
:1004600093022000E31252FEB74E0000130E00026A
:10047000639ED119130200009300100013000000C6
:10048000130000001301F001B391200013021200C9
:1004900093022000E31252FEB70E0080130E1002EA
:1004A0006396D1171302000013017000930010002F
:1004B000B39120001302120093022000E31652FEB3
:1004C000930E0008130E20026392D1151302000050
:1004D0001301E0009300100013000000B39120000E
:1004E0001302120093022000E31452FEB74E0000E4
:1004F000130E3002639CD111130200001301F001AE
:10050000930010001300000013000000B3912000BE
:100510001302120093022000E31252FEB70E008075
:10052000130E40026394D10F1302000013017000F8
:100530001300000093001000B3912000130212007A
:1005400093022000E31452FE930E0008130E500293
:10055000639ED10B130200001301E00013000000A2
:100560009300100013000000B3912000130212004A
:1005700093022000E31252FEB74E0000130E6002F9
:100580006396D109130200001301F001130000006B
:100590001300000093001000B3912000130212001A
:1005A00093022000E31252FEB70E0080130E700279
:1005B000639ED1059300F00033111000930E0000EC
:1005C000130E80026314D1059300000233910000E2
:1005D000930E0002130E9002631AD103B3100000B1
:1005E000930E0000130EA0026392D003930000400C
:1005F000371100001301018033902000930E00009A
:10060000130EB0026314D001631CC0010F00F00F81
:1006100063000E00131E1E00136E1E007300000008
:100620000F00F00F130E100073000000731000C0D5
:1006300000000000000000000000000000000000BA
:0406400000000000B6
:1010000000000000000000000000000000000000E0
:1010100000000000000000000000000000000000D0
:1010200000000000000000000000000000000000C0
:1010300000000000000000000000000000000000B0
:081040000000000000000000A8
:040000058000200057
:00000001FF
